S02B0000433A2F576F726B2F736F6674776172652F4F70656E424C542F5461726765742F44656D6F2F41524DEF
S31508000000E809002051010008A5190008A5190008EB
S31508000010A5190008A5190008A5190008A5190008BA
S31508000020A5190008A5190008A5190008A5190008AA
S31508000030A5190008A5190008A5190008A51900089A
S31508000040A5190008A5190008A5190008A51900088A
S31508000050A5190008A5190008A5190008A51900087A
S31508000060A5190008A5190008A5190008A51900086A
S31508000070A5190008A5190008A5190008A51900085A
S31508000080A5190008A5190008A5190008A51900084A
S31508000090A5190008A5190008A5190008A51900083A
S315080000A0A5190008A5190008A5190008A51900082A
S315080000B0A5190008A5190008A5190008A51900081A
S315080000C0A5190008A5190008A5190008A51900080A
S315080000D0A5190008A5190008A5190008A5190008FA
S315080000E0A5190008A5190008A5190008A5190008EA
S315080000F0A5190008A5190008A5190008A5190008DA
S31508000100A5190008A5190008A5190008A5190008C9
S31508000110A5190008A5190008A5190008A5190008B9
S31508000120A5190008A5190008A5190008A5190008A9
S31508000130A5190008A5190008A5190008A519000899
S31508000140A5190008A5190008A5190008A519000889
S3150800015072B628498D4628482849294A00F039F8B0
S3150800016028482949294A00F034F8294829492A4AB9
S3150800017000F02FF829482A492A4A00F02AF82A487E
S315080001802A492B4A00F025F82A482B492B4A00F021
S3150800019020F82B482B49002200F026F82A482B493C
S315080001A0091A082903DB00220260043001601C4892
S315080001B01C49884205D00268043003B4904703BC42
S315080001C0F7E700208646EC4600200021204A9047A3
S315080001D0FEE7884207D0521A05D0037801300B7023
S315080001E00131013AF9D17047884202D002700130D4
S315080001F0FAE77047E8090020B42D0008000000203F
S31508000200F00000205402000854020008F82A0008EA
S31508000210B42D00080000002000000020F82A00087D
S31508000220F82A0008F82A0008F82A0008F82A000818
S31508000230F82A0008F82A0008F82A0008B42D000849
S31508000240F00000206807002068070020E807002063
S30908000250F50200089D
S31508000254C0B240F2F003C2F200031B78D3B94FF4DC
S315080002648053C4F202039A6942F010029A614FF469
S315080002748053C4F201035A6822F470425A605A68D9
S3150800028442F4E0425A6040F2F003C2F200034FF02F
S3150800029401021A7001284FF48053C4F201034FF483
S315080002A400620CBF5A611A61704700BF4FF480534D
S315080002B4C4F202039A6942F004029A614FF4006395
S315080002C4C4F201031A6822F00F021A601A6842F08F
S315080002D404021A60704700BF4FF40063C4F20103B6
S315080002E49B6813F0010F14BF00200120704700BF5C
S315080002F400B582B04FF00003009301934FF4805386
S31508000304C4F202031A6842F001021A6059684FF0EF
S315080003140002CFF6FF020A405A601A6822F0847275
S3150800032422F480321A601A6822F480221A605A6803
S3150800033422F4FE025A604FF41F029A601A6842F4C5
S3150800034480321A604FF48053C4F2020340F2DC523E
S31508000354196801F400310191009901F10101009134
S31508000364019911B900999142F2D14FF48053C4F21C
S3150800037402031B6813F4003F04D12E484FF06C01A6
S3150800038402F0CCF84FF40053C4F202031A6842F0A0
S3150800039410021A601A6822F003021A601A6842F0F8
S315080003A402021A604FF48053C4F202035A685A6070
S315080003B45A6842F400525A605A6842F480625A6093
S315080003C45A6822F47C125A605A6842F4E8125A604F
S315080003D41A6842F080721A604FF48053C4F202031A
S315080003E41A6812F0007FFBD04FF48053C4F202035C
S315080003F45A6822F003025A605A6842F002025A60A6
S315080004044FF48053C4F202035A6802F00C02082A15
S31508000414FAD14FF48053C4F202035A6822F48002D4
S315080004245A60DA6942F40002DA6102F091F802F0DD
S315080004349DF8FCE7F82A000800B580B248B940F2EE
S315080004442413C2F200031B684FF001021A835DF8F5
S3150800045404FB40F22813C2F200031B681B68984782
S3150800046440F22413C2F20003186800F112005DF882
S3150800047404FB00BF00B580B248B940F22413C2F2A7
S3150800048400031B684FF001021A835DF804FB40F26F
S315080004942813C2F200031B689B68984740F224138A
S315080004A4C2F20003186800F114005DF804FB00BFEB
S315080004B400B580B248B940F22413C2F200031B689F
S315080004C44FF002021A835DF804FB40F2F803C2F205
S315080004D400034FF000021A8040F22413C2F200030C
S315080004E41A68137813F07F031BD1537C13F0200F7B
S315080004F440F2F802C2F20002117814BF41F0020178
S3150800050421F00201117013F0400F40F2F803C2F211
S3150800051400031A7814BF42F0010222F001021A708D
S3150800052431E0012B3CD0022B40D1537A03F00F0261
S3150800053413F0800F13D04FEA820202F1804202F5CB
S31508000544B842136803F03003102B1CD140F2F803A9
S31508000554C2F200031A7842F001021A7013E04FEA55
S31508000564820202F1804202F5B842136803F440534A
S31508000574B3F5805F07D140F2F803C2F200031A7894
S3150800058442F001021A7040F22813C2F200031B68F3
S315080005941B69984740F2F800C2F200005DF804FBB4
S315080005A440F2F800C2F200005DF804FB4FF00000C8
S315080005B45DF804FBF0B540F22413C2F200031C688C
S315080005C4238B227C8BBB042A64D140F2F403C2F247
S315080005D400031B68012B1ED145F65043C4F20003E1
S315080005E41A6892B243F20203C2F20003D3184FEA1E
S315080005F443034FF000021A6040F23613C2F20003B6
S315080006044FF03001198040F2F403C2F200031A6075
S315080006144FF0040637E040F23613C2F200034FF0F7
S3150800062410021A804FF007062DE0A58BAB428CBF4B
S31508000634022604269D4228BF1D46236A2846984753
S3150800064407464FF0000000F06BFF014638462A467D
S3150800065400F04CFE4FF00000294600F085FF238B7E
S315080006645B1B2383638BED18658340F23613C2F252
S3150800067400034FF030021A8040F23413C2F200032A
S315080006844FF440521A8040F22413C2F200031B6846
S315080006941E74F0BDA58B4FF00406CBE700B540F2F7
S315080006A42413C2F200031A68517940F2E803C2F22D
S315080006B400035B788B420FD313798BB913899BB9E3
S315080006C4917440F22813C2F200031B685B689847CA
S315080006D44FF000005DF804FB4FF002005DF804FBE0
S315080006E44FF002005DF804FB4FF002005DF804FBCE
S315080006F410B540F22414C2F20004226840F2301302
S31508000704C2F200031B68507A51799B69984723689B
S315080007149A7C9AB1A8B91A7AB2B91B79BBB940F2CC
S315080007242813C2F200031B68DB68984723685A7AC1
S31508000734DA745A791A754FF0000010BD4FF00200AA
S3150800074410BD4FF0020010BD4FF0020010BD4FF06F
S31508000754020010BD10B540F22413C2F200031A6851
S31508000764137813F07F0306D1537C23F020035374C4
S315080007744FF0000010BD022B70D19388002B70D166
S31508000784137A002B70D1507A20F0800110F0800F74
S315080007944FEA810303F1804303F5B84319BF1C6884
S315080007A404F030041B6803F4405440F2E803C2F230
S315080007B400031B7899425AD2002C5BD0937C002BF9
S315080007C45BD010F0800F14D04FEA810303F1804305
S315080007D403F5B8431B6803F03003102B37D1CCB2AA
S315080007E4204600F05DFE20464FF0300100F0CCFDB7
S315080007F42DE04FEA810404F1804404F5B8442368E3
S3150800080403F44053B3F5805F21D191B91C4B93F897
S315080008142C104FF0000000F0BBFE22684BF68F73D5
S31508000824134083F4405343F4004343F080032360A6
S315080008340DE0C8B200F01EFE22684BF68F73134013
S3150800084483F4405343F4004343F0800323600D4B81
S315080008541B685B6998474FF0000010BD4FF0020013
S3150800086410BD4FF0020010BD4FF0020010BD4FF04E
S31508000874020010BD4FF0020010BD4FF0020010BD7B
S315080008845C0000202801002010B540F22413C2F2AF
S3150800089400031868427A22F0800112F0800F4FEAAA
S315080008A4810303F1804303F5B84319BF1C6804F0B8
S315080008B430041B6803F4405440F2E803C2F2000310
S315080008C41B78994237D28388002B37D1002C38D02D
S315080008D4837C002B38D012F0800F11D04FEA8102A6
S315080008E402F1804202F5B842116848F6BF730B401C
S315080008F483F0100343F4004343F08003136010E0CD
S315080009044FEA810202F1804202F5B84211684BF6B9
S315080009148F730B4083F4805343F4004343F08003FE
S31508000924136040F22813C2F200031B689B699847B8
S315080009344FF0000010BD4FF0020010BD4FF002004A
S3150800094410BD4FF0020010BD4FF0020010BD00BFED
S3150800095400B540F22413C2F200031B685A7C42F025
S3150800096420025A7440F22813C2F200031B68DB699A
S3150800097498474FF000005DF804FB00BF80B240F2D0
S315080009842413C2F200031B685A8B28B98888821A72
S315080009941A834FF00000704708688018704700BF34
S315080009A400B540F25C03C2F2000393F82C104FF032
S315080009B4000000F0EDFD40F22413C2F200031B68A8
S315080009C4187C08280DD140F23413C2F200034FF400
S315080009D480521A8040F23613C2F200034FF0100216
S315080009E41A80092814BF002001205DF804FB00BF03
S315080009F470B540F22413C2F200031C68237C022B50
S31508000A047DD0042B7ED0032B01D0052B6BD1228BF2
S31508000A14236AB3B1AAB1A58B954228BF15462846C1
S31508000A2498470646238B5B1B2383638BEB186383E8
S31508000A344FF0000000F086FD014630462A4600F0D5
S31508000A4471FC238B93B140F23413C2F200034FF4C2
S31508000A5440521A804FF00000014600F085FD40F22E
S31508000A643613C2F200034FF030021A80238BA28B8E
S31508000A749A4208D840F22413C2F200031B684FF0C6
S31508000A8403021A7428E043B140F22413C2F20003A5
S31508000A941B684FF005021A741EE040F22413C2F2D2
S31508000AA400031B684FF006021A7445F65043C4F255
S31508000AB400031A6892B243F20203C2F20003D3187F
S31508000AC44FEA43034FF000021A6040F23613C2F2AB
S31508000AD400034FF030021A8040F22413C2F20003D6
S31508000AE41B681A7C13E0072B0FD140F23013C2F2AD
S31508000AF400031B68DB6898474FF0080207E04FF0CD
S31508000B04080204E04FF0080201E04FF0080240F240
S31508000B142413C2F200031B681A74FFF741FF70BD61
S31508000B2470B581B045F65043C4F200031A6892B210
S31508000B3443F20403C2F20003D3184FEA43031D68C1
S31508000B4440F22413C2F200031B681A7C092A1CD03B
S31508000B54ADB205F1005505F540554FEA45052A7825
S31508000B641A7040F22414C2F2000423686A785A7090
S31508000B742668A88800F04EFDB0802668288900F00B
S31508000B8449FD3081AA8923689A8140F22413C2F266
S31508000B9400031B684FF001021A749989002940F072
S31508000BA482805C781A7812F07F022CD1092C02D143
S31508000BB4FFF774FD39E0052C0DD193F90520002AB9
S31508000BC459DB1A79002A59D11A89002A59D19B7CEA
S31508000BD4002B36D058E0032C07D15A79012A25D19F
S31508000BE41B891BBBFFF7B4FE1FE0012C1ED15A79E3
S31508000BF4012A1BD11A89CAB95B7C13F0200F15D0B8
S31508000C04FFF7A8FD11E0012A04D10B2C0ED1FFF73A
S31508000C146FFD0AE0022A09D1012C02D1FFF79AFDD9
S31508000C2403E0032C02D1FFF72FFE50B140F2301334
S31508000C34C2F200031B685B6920469847032826D03E
S31508000C4440BB45F65043C4F200031A6892B243F215
S31508000C540203C2F20003D3184FEA43034FF000021B
S31508000C641A6040F23613C2F200034FF030021A80BB
S31508000C744FF0060210E04FF008020DE04FF00802AC
S31508000C840AE04FF0080207E04FF0080204E04FF0CC
S31508000C94090201E04FF0080240F22413C2F20003ED
S31508000CA41B681A740EE15A78062A20D11A7812F0AB
S31508000CB47F0F40F094801B79012B06D140F2301344
S31508000CC4C2F200031B68DB697CE0022B06D140F202
S31508000CD43013C2F200031B681B6A73E0032B7ED130
S31508000CE440F23013C2F200031B685B6A6AE0002A0A
S31508000CF446D19888002843D1022941D1187A002878
S31508000D043ED11A7812F07F0204D11989002900F01D
S31508000D14DD8014E0012A12D140F23012C2F2000238
S31508000D241268587A93694FF000019847002856D1FB
S31508000D346E4B1B689B7C002B40F0CD804FE0022A4B
S31508000D444DD15A7A02F00F0112F0800F4FEA81034F
S31508000D5403F1804303F5B843186814BF00F0300064
S31508000D6400F4405040F2E803C2F200031B789942AB
S31508000D7435D212F0700F32D1002840F0AE802EE042
S31508000D84082A05D11B7813F07F0F00F0A88026E007
S31508000D940A2A24D11A7802F07F02012A1FD19A7CE2
S31508000DA4EAB19A88DAB91A7ACAB9012917D1504A1E
S31508000DB41268587A93694FF000019847002800F0A2
S31508000DC493800CE05BB140F22412C2F2000212686E
S31508000DD44FF00004548313622046984718E040F203
S31508000DE43013C2F200031A6840F22413C2F2000355
S31508000DF41B685878136998470446032808D140F2B3
S31508000E042413C2F200031B684FF009021A7459E04E
S31508000E1440F22413C2F200031B681A8B4FF6FF71C3
S31508000E248A4203D14FF009021A744BE0022C00D00F
S31508000E341AB94FF008021A7444E093F9001000290D
S31508000E4436DA998900910098824202D9009A1A835F
S31508000E541EE08A421CD240F23013C2F200031B6819
S31508000E6493F82C309A4207D240F2F403C2F20003F4
S31508000E744FF000021A600BE092FBF3F103FB112317
S31508000E8433B940F2F403C2F200034FF001021A60C8
S31508000E9440F22413C2F200031A6840F23013C2F275
S31508000EA400031B6893F82C309383FFF783FB09E050
S31508000EB44FF003021A7440F23413C2F200034FF4DB
S31508000EC440521A80FFF76CFD01B070BD40F2B5437D
S31508000ED4C0F6000377E7074B75E7064B73E740F25E
S31508000EE43D43C0F600036EE7034B6CE7240100207C
S31508000EF430010020B50400087904000870B4C0B2B3
S31508000F0440F2E803C2F200031D78B5B14FF00003BE
S31508000F1440F60F76DAB24FEA820101F1804101F513
S31508000F24B8410C6842F4004242F08002344022433D
S31508000F340A6003F101039D42ECD840F0800045F6AF
S31508000F444C43C4F20003186070BC704700B540F205
S31508000F542413C2F200031A68137C022B01D0042B53
S31508000F6408D1FFF727FB40F22413C2F200031B68DB
S31508000F741A7C1EE0062B1AD15378052B0DD113784B
S31508000F8413F07F0F09D15079FFF7B8FF40F2281301
S31508000F94C2F200031B681B6A984740F23013C2F278
S31508000FA400031B689B6898474FF0080201E04FF05E
S31508000FB4080240F22413C2F200031B681A74FFF7EE
S31508000FC4EFFC5DF804FB00BF704700BF00B540F2B4
S31508000FD42412C2F2000240F2FC03C2F200031360B8
S31508000FE44FF002021A7440F23012C2F2000240F2C2
S31508000FF45C03C2F20003136040F22812C2F2000234
S3150800100440F28C01C2F2000111601B6898475DF832
S3150800101404FB00BF30B581B04FF00003ADF80230D1
S3150800102440F23A14C2F2000440F22015C2F2000556
S315080010344EE1238803F00F032B70002B40F00F8139
S315080010444FF4B842C4F20002116889B240F234136C
S31508001054C2F200031980188800F0300040F23611F5
S31508001064C2F200010880198801F4405119801168F8
S315080010744BF6BF730B4083F4005383F0200343F409
S31508001084004343F080031360238813F0100F46D1FE
S315080010944FF4B844C4F20004226848F60F731340A8
S315080010A42360FFF753FF22684BF6BF73134040F2E1
S315080010B43412C2F20002128802F4805292B20AB1C1
S315080010C483F4805340F23412C2F20002128802F406
S315080010D4005292B20AB183F4005340F23612C2F2B5
S315080010E40002128802F0100292B20AB183F01003C9
S315080010F440F23612C2F20002128802F0200292B2BC
S315080011040AB183F0200348F28002CFF6FF721A432D
S3150800111492B24FF4B843C4F200031A60E3E04FF402
S31508001124B843C4F200031B689BB2ADF80230BDF89D
S31508001134023013F4006F46D04FF4B844C4F20004E6
S31508001144226840F68F7313402360FFF7E9FC226890
S315080011544BF6BF73134040F23412C2F200021288EF
S3150800116402F4805292B20AB183F4805340F23412E4
S31508001174C2F20002128802F4005292B20AB183F44F
S31508001184005340F23612C2F20002128802F010022C
S3150800119492B20AB183F0100340F23612C2F2000288
S315080011A4128802F0200292B20AB183F0200348F2B0
S315080011B48002CFF6FF721A4392B24FF4B843C4F2D0
S315080011C400031A608FE0BDF802301BB2002B7FDAE9
S315080011D44FF4B844C4F20004226840F68F731340EF
S315080011E42360FFF705FC22684BF6BF73134040F2F1
S315080011F43412C2F20002128802F4805292B20AB180
S3150800120483F4805340F23412C2F20002128802F4C4
S31508001214005292B20AB183F4005340F23612C2F273
S315080012240002128802F0100292B20AB183F0100387
S3150800123440F23612C2F20002128802F0200292B27A
S315080012440AB183F0200348F28002CFF6FF721A43EC
S3150800125492B24FF4B843C4F200031A6043E04FEA6B
S31508001264830303F1804303F5B8431A6892B2ADF8D1
S315080012740220BDF8022012B2002A0EDA196840F6D6
S315080012848F720A401A6040F23803C2F200032A78C1
S3150800129402F1FF3253F822309847BDF8023013F0B2
S315080012A4800F15D02A784FEA820202F1804202F5AD
S315080012B4B842116848F60F730B40136040F21C03DA
S315080012C4C2F200032A7802F1FF3253F82230984713
S315080012D445F64443C4F200031B689BB2238013F407
S315080012E4004F7FF4A6AE01B030BD00BF30B489B25A
S315080012F492B202F10102521011D001F1005101F526
S3150800130440554FEA45054FF00003447810F8021B90
S3150800131441EA0421595303F10403013AF5D130BCD7
S31508001324704700BF10B489B292B202F1010252109A
S315080013340ED001F1005101F540514FEA41014FF039
S31508001344000351F8044BC45203F10203013AF8D1DD
S3150800135410BC70474FF6F873034045F65042C4F282
S3150800136400021360704700BFC0B289B24FEA80001A
S3150800137400F1804000F5B840026848F68F13134020
S315080013840B430360704700BFC0B289B24FEA8000BE
S3150800139400F1804000F5B840026848F6BF73134070
S315080013A401F0100292B20AB183F0100301F0200191
S315080013B489B209B183F0200343F4004343F0800360
S315080013C403607047C0B289B24FEA800000F18040DA
S315080013D400F5B84002684BF68F73134001F4805247
S315080013E492B20AB183F4805301F4005189B209B167
S315080013F483F4005343F4004343F0800303607047C7
S31508001404C2B24FEA820202F1804202F5B84211687A
S3150800141448F6BF730B4083F0300343F4004343F0AC
S3150800142480031360704700BFC2B24FEA820202F11A
S31508001434804202F5B84211684BF68F730B4083F469
S31508001444405343F4004343F080031360704700BFDE
S31508001454C2B24FEA820202F1804202F5B84211682A
S3150800146440F60F630B4043F4004343F080031360D4
S31508001474704700BFC3B24FEA830303F1804303F501
S31508001484B8431A6812F4804F08D0196840F60F72E8
S315080014940A4042F4404242F080021A60704700BF94
S315080014A4C3B24FEA830303F1804303F5B8431A68CA
S315080014B412F0400F08D0196840F60F720A4042F439
S315080014C4004242F0C0021A60704700BFC0B245F637
S315080014D45043C4F200031A6892B202EBC00202F146
S315080014E4005202F540524FEA42024FF6FE730B4091
S315080014F413607047C0B245F65043C4F200031B6834
S315080015049BB203EBC00043F20403C2F20003C31800
S315080015144FEA43034FF6FE720A401A60704700BF4B
S31508001524C0B245F65043C4F200031B689BB203EBF2
S31508001534C00303F1005303F540534FEA43031888E5
S31508001544704700BFC0B245F65043C4F200031B6897
S315080015549BB203EBC00043F20403C2F20003C318B0
S315080015644FEA430318887047C0B289B245F6504318
S31508001574C4F200031B689BB203EBC00043F20203E8
S31508001584C2F20003C3184FEA43031960704700BF49
S31508001594C0B289B245F65043C4F200031B689BB235
S315080015A403EBC00043F20603C2F20003C3184FEA72
S315080015B443033E290DD94FEA511211F01F0F04BFF8
S315080015C402F1FF3292B24FEA822242F400421A60D2
S315080015D470474FEA510211F0010F18BF01324FEA62
S315080015E482221A60704700BFC0B245F65043C4F25F
S315080015F400031B689BB203EBC00043F20603C2F266
S315080016040003C3184FEA430318684FEA80504FEAA9
S315080016149050704780B2C3B24FEA102040EA0320C4
S31508001624704700BF45F64443C4F200034FF0000078
S31508001634186040F22C13C2F200034FF406421A80D3
S3150800164445F64043C4F200031A60704770B50E4667
S3150800165400F07F052846FFF7C7FF04462846FFF72C
S3150800166471FF014630462246FFF75CFE204670BDF0
S3150800167400B500F0A3FE5DF804FB00BF00B500F05A
S31508001684FBFE5DF804FB00BF00B540F23C13C2F252
S3150800169400031B68052B01D100F090FE5DF804FBDE
S315080016A400B545F64443C4F200031A6892B240F200
S315080016B43A13C2F200031A801A8840F22C13C2F2B3
S315080016C400031B88134013F4007F11D045F64443E6
S315080016D4C4F200034FF6FF521A6040F23813C2F2FE
S315080016E400031A7802F10102D2B21A70FFF7CCFF8E
S315080016F440F23A13C2F200031A8840F22C13C2F2DB
S3150800170400031B88134013F4004F01D0FFF782FC33
S3150800171440F23A13C2F200031A8840F22C13C2F2BA
S3150800172400031B88134013F4806F0CD045F644431A
S31508001734C4F200034FF6FF321A6040F25C03C2F2A9
S3150800174400035B6898475DF804FB00BF40F2FC039E
S31508001754C2F200039B7C33B140F23C13C2F200038D
S315080017644FF005021A60704740F23C13C2F20003B8
S315080017744FF004021A607047704700BF704700BFF5
S3150800178410B5C0B2062811D140F22413C2F20003E0
S315080017941B681A7802F07F02012A0AD15A7A5AB9C2
S315080017A41A79212A0BD04FF0020010BD4FF002001F
S315080017B410BD4FF0020010BD4FF0020010BD41F2FB
S315080017C4FD72C0F600021A624FF000045C832046DC
S315080017D400F012F8204610BD4FF00200704700BF13
S315080017E4C0B2C9B221B9002814BF0220002070472C
S315080017F44FF00200704700BF00B580B240F2B00156
S31508001804C2F20001FFF7BAF85DF804FB00B580B22E
S3150800181440F22413C2F200031B685B79052B09D82E
S3150800182440F2C001C2F2000101EBC301FFF7A6F8BA
S315080018345DF804FB4FF000005DF804FB00B580B2C8
S3150800184440F25401C2F20001FFF798F85DF804FB70
S3150800185400B580B240F2B801C2F20001FFF78EF873
S315080018645DF804FB10B540F22413C2F200031B68AA
S315080018744FF000049C7442F69C32C0F60002D279FA
S315080018845A74DC742046FFF765FD20464FF4007150
S31508001894FFF76AFD20464FF01001FFF775FD204655
S315080018A44FF04001FFF726FE20464FF08001FFF770
S315080018B40DFE2046FFF7CCFD40F25C03C2F200039E
S315080018C493F82C102046FFF763FE2046FFF7ACFD7D
S315080018D44FF001002146FFF747FD4FF001004FF492
S315080018E48071FFF7F3FD4FF001004FF0C001FFF7D9
S315080018F401FE4FF001004FF04001FFF735FE4FF0AF
S3150800190401004FF04001FFF743FE4FF001004FF48A
S315080019144051FFF757FD4FF001004FF02001FFF744
S3150800192433FD2046FFF7EAFA40F23C13C2F20003FD
S315080019344FF001021A6010BD10B500F0CDFD40F25B
S315080019442413C2F200031B684FF000049C7400F0D1
S3150800195409F8FFF767FE40F23C13C2F200031C6065
S3150800196410BD00BF00B54FF00100FEF771FC45F647
S315080019744043C4F200034FF001021A6040F22C12ED
S31508001984C2F200024FF00000186045F64441C4F262
S31508001994000108604FF4E051118019605DF804FBFA
S315080019A400B542F60440C0F600004FF03D0100F0D1
S315080019B4B5FD5DF804FB00BF00B500F03DF890B135
S315080019C400F006FE00F050F800F03CF820F0604005
S315080019D420F07F004EF60853CEF20003186000F09C
S315080019E431F8436898475DF804FB00BF70B50E46A6
S315080019F492B272B1044600F1010002F1FF3292B2CA
S31508001A04851816F8013B04F8013B00F025FEAC42A4
S31508001A14F7D170BD00B500F0ADF95DF804FB00BF61
S31508001A2400B500F0B5F95DF804FB00BF00B500F099
S31508001A34DBF95DF804FB00BF00B500F0A3FA5DF816
S31508001A4404FB00BF00B500F0FDFA5DF804FB00BF17
S31508001A5400B500F069FA18B100F0C8FA5DF804FB9D
S31508001A644FF000005DF804FB4EF21003CEF20003BB
S31508001A744FF000021A60704700B5FFF7F5FF4EF203
S31508001A841003CEF2000341F63F12C0F201025A6077
S31508001A944FF000029A604FF00501196040F24013B6
S31508001AA4C2F200031A605DF804FB00BF4EF210038D
S31508001AB4CEF200031B6813F4803F07D040F24013AC
S31508001AC4C2F200031A6802F101021A60704700BFE5
S31508001AD44FF40053C4F2020340F22312C4F26752CD
S31508001AE45A6048F6AB12CCF6EF525A604FF03402FD
S31508001AF4DA6070474FF40053C4F202031A6942F0DD
S31508001B0480021A61704700BF70B5064642F69045D2
S31508001B14C0F600054FF0000400F09EFD2B68B342A2
S31508001B240DD869685B189E4209D242F69043C0F6FE
S31508001B34000304EB440203EB8203187A70BD04F134
S31508001B44010405F10C050D2CE6D14FF0FF0070BD1C
S31508001B542DE9F04107460068FFF7D6FFFF2855D060
S31508001B64FFF7B6FF4FF40053C4F20203DB6813F021
S31508001B74010F04D0FFF7BEFF4FF0000448E04FF40E
S31508001B840053C4F202031A6942F001021A614FF0C3
S31508001B9400054FF40054C4F202043B6805EB03083D
S31508001BA405F10402BE58B2B2EA52E36813F0010F13
S31508001BB405D000F051FDE36813F0010FF9D14FEA9F
S31508001BC41643A8F80230E36813F0010F05D000F0B5
S31508001BD443FDE36813F0010FF9D1D8F80030B34296
S31508001BE407D105F10405B5F5007FD6D14FF00104F8
S31508001BF401E04FF000044FF40053C4F202031A69DB
S31508001C0422F001021A61FFF775FF01E04FF00004A4
S31508001C142046BDE8F08100BF70B5C6B242F69045CD
S31508001C24C0F600054FF0000400F016FD2B7AB34207
S31508001C3408D142F69043C0F6000304EB440253F875
S31508001C44220070BD04F1010405F10C050D2CEBD13D
S31508001C544FF0FF3070BD00BF00B54FEAC1534FEADD
S31508001C64D35363B903688B420DD040F8041B4FF471
S31508001C740072FFF7BBFE4FF001005DF804FB4FF05E
S31508001C8400005DF804FB4FF001005DF804FB00BF9B
S31508001C9430B504460D4640F24413C2F20003984296
S31508001CA409D04FF4C043C0F60003994208D0FFF7A1
S31508001CB44FFF48B910E040F24834C2F2000403E08A
S31508001CC440F24414C2F2000420462946FFF7C4FF32
S31508001CD4002808BF002401E04FF00004204630BD68
S31508001CE42DE9F04305460C4617461E464FEA512988
S31508001CF44FEA49290368B3F1FF3F03D14946FFF781
S31508001D04ABFF50B32B684B4505D028464946FFF729
S31508001D14BFFF054628B32B68E41A04F104042C19FA
S31508001D2440F2FF1809F5007900F096FC05F1040362
S31508001D34E31A434507D928464946FFF7A9FF054646
S31508001D4498B100F1040417F8013B04F8013B013E7D
S31508001D54EAD14FF00100BDE8F0834FF00000BDE87A
S31508001D64F0834FF00000BDE8F0834FF00000BDE8B3
S31508001D74F08300BF40F24833C2F200034FF0FF324B
S31508001D841A6040F24413C2F200031A60704700BF97
S31508001D9470B504460D461646FFF7B6FEFF281DD055
S31508001DA404F1FF304019FFF7AFFEFF2819D04FEAB8
S31508001DB454224FF4C043C0F60003B3EB422F07BFC7
S31508001DC440F24410C2F2000040F24830C2F2000069
S31508001DD4214632462B46FFF783FF70BD4FF00000BD
S31508001DE470BD4FF0000070BD2DE9F04104460E4663
S31508001DF4FFF78AFE054604F1FF34A019FFF784FEAF
S31508001E0404460646FF2D00F08780FF2800F08880E8
S31508001E14854275D8022D77D90F2879D8FFF758FE49
S31508001E244FF40053C4F20203DB6813F0010F05D024
S31508001E34FFF760FE4FF00000BDE8F0814FF4005351
S31508001E44C4F202031A6942F002021A612846FFF72D
S31508001E54E3FE07462046FFF7DFFE804642F6904536
S31508001E64C0F600054FF0000400F0F6FB2B7AB342E7
S31508001E7409D142F69043C0F6000304EB440203EB8F
S31508001E8482035B6807E004F1010405F10C050D2CD7
S31508001E94EAD14FF00003C7EB08084344C3F38F2382
S31508001EA403B303F1FF339EB206F101064FEA862611
S31508001EB44FF000054FF40054C4F20204EB196361B1
S31508001EC4236943F040032361E36813F0010F05D047
S31508001ED400F0C2FBE36813F0010FF9D105F580653C
S31508001EE4B542EBD14FF40053C4F202031A6922F047
S31508001EF402021A61FFF7FEFD4FF00100BDE8F0810A
S31508001F044FF00000BDE8F0814FF00000BDE8F08115
S31508001F144FF00000BDE8F0814FF00000BDE8F08105
S31508001F244FF00000BDE8F08100B581B040F24413DB
S31508001F34C2F200031B68B3F1FF3F1FD040F24413FB
S31508001F44C2F2000399685A688918DA6889181A69FE
S31508001F5489185A6989189A698918DA698B18C3F12C
S31508001F64000301AA42F8043D46F25010C0F60000E8
S31508001F744FF004016A46FFF70BFF01E04FF001003A
S31508001F8401B000BD46F20402C0F600024FF4C04395
S31508001F94C0F6000310681B68C01846F20803C0F6AA
S31508001FA400031B68C01846F20C03C0F600031B683E
S31508001FB4C01846F21003C0F600031B68C01846F2A0
S31508001FC41403C0F600031B68C01846F21803C0F6CB
S31508001FD400031B68C01846F25013C0F600031B68BA
S31508001FE4C018D0F1010038BF0020704700B540F290
S31508001FF44413C2F200031B68B3F1FF3F06D040F254
S315080020044410C2F20000FFF7A3FD90B140F2483332
S31508002014C2F200031B68B3F1FF3F0ED040F248300A
S31508002024C2F20000FFF794FD003018BF01205DF8E6
S3150800203404FB4FF000005DF804FB4FF001005DF867
S3150800204404FB00BF4FF4C040C0F60000704700BF51
S3150800205410B4D2B2BAB10B4601F1020102F1FF3251
S31508002064D2B201EB42014FF000044FEA1072092A7A
S3150800207494BF303237321A704FEA00105C7003F19D
S3150800208402038B42F1D110BC704700BF10B4C9B229
S3150800209440F2D053C2F200031B6893B140F2D05207
S315080020A4C2F200025C69146019749860D8604FF033
S315080020B400025A74186001F1FF3140185860987C80
S315080020C401E04FF0FF0010BC704700BF30B5C4B242
S315080020D4CDB2012C07D942F62C50C0F6000040F2C6
S315080020E4FD1100F01BFA40F2D453C2F2000304EBCC
S315080020F4440203EBC2035A7C1B7C9A4222D040F268
S31508002104D453C2F2000304EB440203EBC203DA68B5
S315080021141570597C01F101015974DA6802F101025A
S31508002124DA605B689A4210D940F2D453C2F20003CB
S3150800213404EB44044FEAC4041A191B59D3604FF03C
S31508002144010030BD4FF0000030BD4FF0010030BD36
S3150800215400B5C1B240F28863C2F200031878FFF7EB
S31508002164B5FF5DF804FB00BF30B50D46C4B2012CBB
S3150800217407D942F62C50C0F6000040F21F2100F0A1
S31508002184CDF940F2D453C2F2000304EB440203EB44
S31508002194C2035B7C0BB340F2D453C2F2000303EBD5
S315080021A4C2039A6812782A70597C01F1FF3159746E
S315080021B49A6802F101029A605B689A4210D940F261
S315080021C4D453C2F2000304EB44044FEAC4041A19B4
S315080021D41B5993604FF0010030BD4FF0000030BD2D
S315080021E44FF0010030BD00BF00B5014640F204635C
S315080021F4C2F200031878FFF7B7FF5DF804FB00BFC7
S3150800220430B540F2D453C2F200034FF000029A7478
S3150800221403F1180159614FF0010183F82A10DA62B3
S3150800222440F2D052C2F20002136040F28864C2F24D
S31508002234000460184FF04001FFF728FF207040F2B1
S315080022440465C2F2000505F101004FF04001FFF7ED
S315080022541DFF28702378FF2B01D0FF2807D142F6EB
S315080022642C50C0F600004FF07F0100F057F9FEF736
S31508002274ADFE30BD00B54FF00000FDF7E9FF5DF88F
S3150800228404FB00BF2DE9F0410546CCB23F2C07D923
S3150800229442F62C50C0F600004FF09E0100F03EF9BD
S315080022A42046FFF755FF012807D042F62C50C0F602
S315080022B400004FF0A20100F031F92646BCB14FF0F8
S315080022C4000442F62C57C0F600074FF0AB0800F09E
S315080022D4C3F9285DFFF73CFF012803D03846414679
S315080022E400F01CF904F10104A3B2B342EFD3BDE82C
S315080022F4F08100BF10B50446FFF7D2F940F2CD537A
S31508002304C2F200031B78EBB940F24C50C2F200004B
S31508002314FFF76AFF012843D140F24C53C2F2000387
S315080023241B78002B3FD040F2CD53C2F200034FF086
S3150800233401021A7040F2CC53C2F200034FF00000B7
S31508002344187010BD40F24C53C2F2000340F2CC524E
S31508002354C2F20002107800F101001818FFF744FFD2
S31508002364012823D140F2CC53C2F200031A7802F1B1
S315080023740102D2B21A7040F24C53C2F200031B781F
S31508002384934216D120460C49FFF730FB40F2CD5351
S31508002394C2F200034FF000021A704FF0010010BD9C
S315080023A44FF0000010BD4FF0000010BD4FF00000C4
S315080023B410BD4FF0000010BD4D0500202DE9F04179
S315080023C481B040F28863C2F200031C78012C07D955
S315080023D442F62C50C0F6000040F23F2100F09EF869
S315080023E440F2D453C2F2000304EB440403EBC403DF
S315080023F45B7C002B3DD0402B34BF98464FF04008F9
S31508002404B8F1000F23D040F28C53C2F2000303F153
S31508002414FF3408F1FF35EDB25D1940F28866C2F261
S31508002424000642F62C57C0F6000730780DF1030172
S31508002434FFF79AFE012804D038464FF4A77100F036
S315080024446DF89DF8033004F8013FAC42EDD140F233
S315080024548C50C2F200004FF480714246FEF746FFE4
S315080024644FF001004146FFF77FF84FF00100FEF7F1
S31508002474C7FF01B0BDE8F081F0B540F24861C2F289
S3150800248400014FF00100FFF7E1F882B2FAB140F219
S315080024944863C2F2000303F1FF3402F1FF3295B236
S315080024A45D1940F20466C2F2000642F62C57C0F6DD
S315080024B40007307814F8011FFFF708FE012804D036
S315080024C4384640F2731100F029F8AC42F1D14FF0C6
S315080024D40100FEF7A9FFF0BD30B54FF2E873C1F667
S315080024E4FF731B684FF2EC72C1F6FF7214684FF261
S315080024F4F072C1F6FF721068C0180CD0064D294652
S315080025044FF00802FFF7A4FD05F1100120464FF02D
S315080025140402FFF79DFD30BD0200002000B540F21D
S31508002524CC63C2F20003186040F2D063C2F200031F
S31508002534196000F091F8FCE700B5FDF7B7FEFDF762
S31508002544CBFE08B9FFF738FA5DF804FB704700BFFD
S3150800255400B500F07FF8FFF78FFAFFF75BFA00F093
S3150800256411F8FFF7E9FF5DF804FB00BF00B500F0BA
S3150800257473F8FFF79BFA00F013F8FFF7E7FF5DF827
S3150800258404FB00BF00B500F07FF8FFF739FE40F200
S31508002594EC03C2F200034FF002021A605DF804FB72
S315080025A400B540F2D460C2F20000FFF7A3FE01288A
S315080025B40CD140F2EC03C2F200034FF002021A6097
S315080025C440F2D460C2F2000000F078F85DF804FB2B
S315080025D400B5FFF74FFE5DF804FB00BF00B589B2EE
S315080025E440F2EC03C2F200031B68022B02D1C9B203
S315080025F4FFF748FE00F058F85DF804FB40F2EC03D8
S31508002604C2F200031A68032A0AD813464FF00102D5
S3150800261402FA03F313F00B0F02D04FF000007047D1
S315080026244FF03F00704700BF40F2EC03C2F20003CC
S315080026341A68032A0AD813464FF0010202FA03F36A
S3150800264413F00B0F02D04FF0000070474FF03F0015
S31508002654704700BF704700BF704700BF40F214734D
S31508002664C2F200034FF000025A70704740F2147326
S31508002674C2F200034FF0FE02DA7018714FF002023C
S31508002684A3F84420704700BF40F21473C2F2000353
S315080026944FF000021A709A6483F84220A3F8442083
S315080026A49A705A70704700BF40F21473C2F200035E
S315080026B44FF0000283F84220704700BF30B5044645
S315080026C40278FF2A23D1FFF7C9FF40F21474C2F235
S315080026D400044FF0010525704FF0FF03E3704FF037
S315080026E4100323714FF000036371FFF787FFA0718E
S315080026F4FFF79AFFE071FFF797FF4FEA1020207261
S315080027046572A5724FF00803A4F84430AEE140F2AE
S315080027141473C2F200031B78012B40F0C981A2F19D
S31508002724C902352A00F29E81DFE812F0F8009C01FE
S315080027349C0197019C019C0189011F016F015901A4
S315080027449C019C019C019C019C019C019C019C018F
S315080027549C019C019C019C019C019C019C019C017F
S315080027649C019C019C019C019C019C019C019C016F
S315080027749C019C019C019C019C019C019C019C015F
S315080027848B00590036007D009C019C019C01B20017
S315080027949C01CE00D300E7004578FFF72FFF00F130
S315080027A4FF30854204DD4FF02200FFF75FFF5DE14D
S315080027B440F21475C2F2000505F10400A96C6278AA
S315080027C4FFF714F94FF0FF03EB706278AB6CD3187C
S315080027D4AB64637803F10103A5F8443046E1457810
S315080027E4FFF70CFF00F1FF30854204DD4FF02200AD
S315080027F4FFF73CFF3AE1616840F21475C2F200053E
S31508002804A96405F104006278FFF7F0F84FF0FF03B6
S31508002814EB706278AB6CD318AB64637803F101038D
S31508002824A5F8443022E140F21473C2F200034FF0D3
S31508002834FF02DA7042689A644FF00102A3F8442052
S3150800284414E140F21473C2F200034FF0FF02DA7087
S31508002854996C436843B14FF0000211F8010B121842
S31508002864D2B2013BF9D101E04FF0000240F21473F1
S31508002874C2F20003C3F807204FF001021A714FF0A1
S3150800288400025A719A714FF00802A3F84420EDE049
S3150800289440F21473C2F200034FF0FF02DA7042F6F4
S315080028A4AC52C0F600029A644FF000021A715A71CB
S315080028B49A714FF00701D9711A725A729A724FF0C7
S315080028C40802A3F84420D1E04FF00000FFF7CEFE3B
S315080028D4CCE040F21473C2F200034FF0FF02DA7040
S315080028E44FF000021A71597859719A71DA711A728D
S315080028F44FF00602A3F84420B8E040F21474C2F27A
S3150800290400044FF000032370FFF7A8FE4FF0FF03FF
S31508002914E3704FF00103A4F84430A7E040F21473BF
S31508002924C2F200039D6CFFF769FE00F1FF3104F162
S3150800293401022846FFF774F820B94FF03100FFF773
S3150800294495FE93E040F21474C2F200044FF0FF03BC
S31508002954E370A56CFFF752FE05F1FF331B18A36459
S315080029644FF00103A4F8443080E04578FFF746FEAB
S31508002974A0F10200854204DD4FF02200FFF776FE3F
S3150800298474E040F21473C2F200034FF0FF02DA70E7
S315080029944FF00102A3F84420617841B9FFF758F8CB
S315080029A4002863D14FF03100FFF760FE5EE040F285
S315080029B41473C2F20003986C04F10202FFF730F8AC
S315080029C420B94FF03100FFF751FE4FE040F214737F
S315080029D4C2F2000361789A6C8A189A6446E040F257
S315080029E41474C2F200044FF0FF03E3704FF00005BD
S315080029F425716571FFF702FEA071E571257265728E
S31508002A044FF00703A4F8443030E040F21473C2F2DE
S31508002A140003986C6168FFF709F820B94FF0310094
S31508002A24FFF724FE22E040F21473C2F200034FF0CB
S31508002A34FF02DA704FF00102A3F8442016E0FEF70D
S31508002A44BBFF40F21473C2F200034FF0FF02DA70C0
S31508002A544FF00102A3F8442008E04FF03100FFF7D5
S31508002A6405FE03E04FF02000FFF700FE40F2147362
S31508002A74C2F2000393F84230012B03D14FF0100041
S31508002A84FFF7F4FD40F21473C2F20003B3F84410DE
S31508002A940BB2002B0CDD40F21470C2F200004FF0AA
S31508002AA4010380F8423000F1030089B2FFF796FD6E
S31508002AB430BD00BF30B504460D4600F017F840F2A5
S31508002AC46073C2F200031D6040F26473C2F200032D
S31508002AD41C601A461368002BFCD100F009F840F272
S31508002AE46073C2F20003186830BD00BF704700BFA8
S30908002AF4704700BF5A
S31508002AF8433A2F576F726B2F736F667477617265D7
S31508002B082F4F70656E424C542F5461726765742F47
S31508002B1844656D6F2F41524D434D335F53544D33C2
S31508002B28325F4F6C696D65785F53544D333248315F
S31508002B3830335F43726F7373776F726B732F426F9D
S31508002B486F742F6964652F2E2E2F6D61696E2E633B
S31508002B58000000001201100100000040501DAC6082
S31508002B6800010102030100000403090426035700B3
S31508002B7869006E00550053004200200042007500A7
S31508002B886C006B002000440065007600690063004D
S31508002B986500000009022000010100C0320904008E
S31508002BA80002FF000004070581024000000705012E
S31508002BB8024000001A034F00700065006E004200CC
S31508002BC84C00540020005500730065007200000090
S31508002BD82C03570069006E00550053004200200078
S31508002BE8420075006C006B00200049006E007400F6
S31508002BF8650072006600610063006500433A2F5756
S31508002C086F726B2F736F6674776172652F4F706575
S31508002C186E424C542F5461726765742F44656D6F04
S31508002C282F41524D434D335F53544D33325F4F6CEA
S31508002C38696D65785F53544D3332483130335F4395
S31508002C48726F7373776F726B732F426F6F742F6916
S31508002C5864652F2E2E2F2E2E2F2E2E2F2E2E2F53E7
S31508002C686F757263652F41524D434D335F53544D0B
S31508002C7833322F43726F7373776F726B732F766560
S31508002C8863746F72732E63000060000800200000EA
S31508002C98030000000080000800200000040000006F
S31508002CA800A00008002000000500000000C0000879
S31508002CB8002000000600000000E0000800200000D0
S31508002CC807000000000001080020000008000000B6
S31508002CD80020010800200000090000000040010843
S31508002CE8002000000A00000000600108002000001B
S31508002CF80B00000000800108002000000C000000FE
S31508002D0800A00108002000000D00000000C001080E
S31508002D18002000000E00000000E001080020000066
S31508002D280F000000433A2F576F726B2F736F667444
S31508002D38776172652F4F70656E424C542F546172D5
S31508002D486765742F44656D6F2F41524D434D335F48
S31508002D5853544D33325F4F6C696D65785F53544DE4
S31508002D683332483130335F43726F7373776F726BE0
S31508002D78732F426F6F742F6964652F2E2E2F2E2E90
S31508002D882F2E2E2F2E2E2F536F757263652F4152B5
S31508002D984D434D335F53544D33322F7573622E634B
S31108002DA8000000004F70656E424C54009D
S31508002DB41C0353004500520031003200330034002E
S31508002DC4350036003700380039003000751600081B
S31508002DD4CD0F0008CD0F0008CD0F0008CD0F000851
S31508002DE4CD0F0008CD0F000881160008CD0F000886
S31508002DF4CD0F0008CD0F0008CD0F0008CD0F000831
S31508002E04CD0F00089C2B0008200000003D1900087F
S31508002E14691800087D170008811700088517000837
S31508002E24DD170008E51700085518000841180008BA
S31508002E34111800080000000040000000CD0F00082B
S31508002E4451170008CD0F0008CD0F0008CD0F000854
S31508002E54CD0F0008CD0F0008CD0F00086D17000828
S31508002E64AE2B0008090000005C2B000812000000C5
S31508002E74702B000804000000BC2B00081A00000090
S31508002E84742B000826000000000000201C00000027
S31508002E94D82B00082C0000000301000004000000E1
S70508000151A0
